:1074000080E189BD82E189BD09B400FEFDCF089508
:10741000AA2069F08091E9008F931092E9007CD452
:1074200083FF01C0FBD48F9187708093E90008959A
:107430008EEF0090E10008220092E1000895F20131
:10744000F999FECFF2BDE1BD0895F9DFF89A80B554
:1074500008C0F5DF1FBA80BD0FB6F894FA9AF99A02
:107460000FBE31962F010895E0E0F0E085919491F0
:10747000019608958BEA3FD0109289008AEF80939D
:10748000880082E080936F0083E08093810098E021
:1074900082E665D0892F877063D08FEF5C9860D0CB
:1074A0009A95B2F7E7E7F7E7859159D0ED37E1F71D
:1074B00081E08093D7008AE482BF1092D8001092B6
:1074C000E2001092DA001092E10080E808D019BCC6
:1074D000AA241092E00036D489E027D481E9809371
:1074E000D8000895A3E6B1E090E812D08D939A9564
:1074F000E1F7089586E008D017C083E005D08F2F0C
:1075000007D08E2F05D080E05B9A90E59CBD5A98FD
:107510008EBD8DB587FFFDCF8EB5089505D085E072
:10752000F3DFF6DF80FDFDCF5A9A88E58CBD5B98CE
:1075300008958FE08221E9F7F7DFE3E6F6E090E0D7
:1075400080E60DD0892F0CD05C98819109D083E61C
:107550008E278F77D1F79395983091F708955C9A9D
:107560005B98D6DF5B9A0895E3E6F1E097FC36C0BE
:1075700094FC4DC092FE089596849920D1F3F8941E
:10758000C089D78520E030E080E090E4AFEFBFEF26
:10759000119689199040E0F72D01BD4F8D0127FD0F
:1075A00013C0E0E0F8E011928EE7819392E4E117D6
:1075B00091939AE508F092E4E334C9F7819310823D
:1075C000BBDFFE01219699DF8DDFF901C9D4205878
:1075D0003F4F040D151D9A9411F701C28301282D08
:1075E00060906C0170906B0143D019F48823C1F74F
:1075F0000895380188243CD0C9F580916A0182172A
:1076000009F4830160906E0170906D01F4CF80E108
:10761000982E60906E0170906D012AD059F48823E5
:10762000B1F708959FEF95FC03C096FE089591E091
:1076300097FB890E662477248301222719D0B1F4A1
:107640008823A1F380916A0136F0881650F48217DE
:1076500030F0213003C0881520F4281710F483017E
:10766000282F60906E0170906D01E8CF3801822E56
:10767000F30143DF37DFC3E6D1E0E0E7F7E7099046
:107680008591081621F4E737D1F7088080104CCF98
:10769000C9E02ADFCA95E9F7D0E197FC55C094FC10
:1076A00037C096FE1AC0C3E6D2E0E3E6F6E098E003
:1076B00088E78E0F00840192E817E1F7884F099060
:1076C0000192E817E1F7C858DF4F9A9589F731DF43
:1076D000C85FD340C33E49F749C0C3E6D6E0EBE5F7
:1076E000FAE098E08E2F885702900086E817E1F7BD
:1076F00038960A900292E817E1F73897C857D040B9
:107700009A9581F716DFC850DC4FC33E41F72EC073
:10771000A3EEB6E0E3E6F6E09AE0C6E00D908081E5
:107720008025807F802582958193A336B90709F44F
:10773000B2E0E336F90709F4F2E0E336FC0771F74B
:10774000F8DEDA9529F712C0A3EEB9E0E3E6FAE035
:1077500092E00E90829180258F70802582958083A3
:10776000E336F907B1F7E5DEDA9571F78827089572
:1077700041524455424F592440486400840000FF60
:10778000FFCFCFFFFFFFFFCFCFFFFF0000FE067E42
:107790007E06FE46565616FE0656461EFE3F61E91A
:0E77A000E3FFE3EBE3FFE3EBE3FFE16B3F000E
:1077AE001201100102000008412336000100000002
:1077BE00000109023E0002010080320904000001AE
:1077CE00020201000524001001042402040524060F
:1077DE000001070582030800FF09040100020A00E8
:1077EE0000000705040210000107058302100001C6
:1078000011241FBE04B714BE88E1E0E6F0E08083D7
:1078100011928EEF9AE09EBF8DBF22243324210166
:107820003101410151018AC00F928F939F931F92A2
:107830000FB60F9211244F936F938091DA0080FF5F
:1078400037C023C00F920FB68F939F93EF93FF9390
:1078500088278093850080938400E0E5F1E09281A1
:10786000907261F490818917980B908309F45D9A66
:1078700091818917980B918309F4289A239411F424
:107880008315381EFF91EF9154C08091D80080FF7E
:107890000FC08091DA008E7F8093DA008091D9004A
:1078A00080FF04C0ADDD81E0A82E02C019BCAA246F
:1078B0008091E10080FF0BC032D280FF08C032D23D
:1078C0008091D80080620BDE19BC85E0A82E8091E3
:1078D000E10084FF1AC023D284FF17C091DD80919C
:1078E000D8008F7DFCDD8FEEA4DD19D28F7E816004
:1078F0001CD280915301882331F48091E30087FDED
:1079000002C081E001C084E0A82E8091E10083FFE5
:107910000CC005D283FF09C087EF8BDD82E0A82E63
:107920001092530185DDFED10DD26F914F910F90D2
:107930001F909F918F910FBE0F90189580E88083C4
:107940001082B1E0B5BF82E085BF81EF85B987EED7
:1079500084B91DB8769A10BA83EF81BB8DE38BB9D9
:107960008FE38AB980E58CBDBDBDA0E0EEEAF7E704
:1079700005900D92A035E1F71D92BB30E9F7599AB9
:1079800004C07C9B02C070DD51F574DD789470DE1C
:1079900071F0ABE9B7E0EDE7F7E790E105900D9204
:1079A0009A95E1F7A059BF4FED3AB9F7C6DD53D02C
:1079B0002FDD80915201807871F48FB18095807FA6
:1079C00066991C9B8460982E2DDE8110CDDD882069
:1079D00011F492FC02C0332052F746DD41F3F894D3
:1079E00089EB89DD81E08093E00010926F001092B6
:1079F0008100109285001092840085BF15BE2E9ADA
:107A0000589A2D9A5D9A289A0C94000083D107C049
:107A100044D102C0AA2039F07FD182FFFBCF85FF7D
:107A2000F7CF8091F1000895082E83E074D185FD91
:107A300007C069D102C0AA2069F06ED180FFFBCFD8
:107A40000092F10080915201807221F45D9884E6E9
:107A50008093500108955ED182FF21C1809152012F
:107A6000807221F4289884E680935101CFDF182F8B
:107A7000853431F422248EE7382EE1DC8DE0F8C025
:107A8000843511F4C3DFFACF8C34C1F38035B1F300
:107A9000843711F480E0ECC0813429F4B7DF582E2C
:107AA000B5DF482EEBCF833539F4E0E7F7E7859172
:107AB000BBDFE737E1F7DDC0863521F482E3B4DFD1
:107AC00081E3D6C0863761F481E3669B8E5F1C9BA1
:107AD0008F5FAADF8FB1809582958F708F5BC8C052
:107AE0008837A9F493DF80935201289A84FD28985F
:107AF0005D9A83FD5D982E9A81FD2E98589A82FD9D
:107B000058982D9A80FD2D9887FD8824B7CF8A3606
:107B100049F48FE9F9DCC3E0FBDC86DFCA95E1F7C5
:107B200003DDA7C0833731F487E87EDF85E97CDF9A
:107B30008EE19EC0823631F489E576DF80E074DF25
:107B400080E896C0823419F0873609F07DC033246E
:107B50005DDFD82F5BDFC82F59DF082F83548430B7
:107B600008F085C0063411F4440C551CF201109243
:107B70006F001736B9F4033489F483E0BFDCC8DC46
:107B80008EB51EBC51DF0DB42197D1F7CDDC08C0F6
:107B9000063411F4859101C058DC46DF2197C2F705
:107BA0002F014AC00334A9F4E11104C0A3DC88ED1D
:107BB000A5DCB4DC9FDC82E0A1DC28DF0DB48EBD47
:107BC000CA95D9F73196A5DCA9DCDA9569F72F01BA
:107BD00031C00634F1F49F01F437D8F4D4D119C080
:107BE00015DF063461F4C0FB46F0F43728F4182E94
:107BF00081E087BFE89511243296082E0AC004342C
:107C000039F4DF01B370AD59B94F8D93319601C08E
:107C100020DC21972AF7043431F42F01F370FE2B76
:107C200049F48BDC07C0063429F42F01F901F4373D
:107C300008F4A7D18DE0F8DE063411F45694479489
:107C400082E080936F0015C08237E1E049F086340E
:107C5000E0E031F08E34E3E019F0813531F4E2E018
:107C6000F0E089E087BF849103C08B3111F08FE38E
:107C7000DBDE83E0DADB47D095FF03C009C0AA2032
:107C800071F04AD080FFFBCF3ED002C0AA2039F06D
:107C900043D080FFFBCF84E0C8DB8BE735C008957D
:107CA000E4E5F1E067E090915B0180915C01913245
:107CB00031F0913A71F5813261F550D173C0823261
:107CC00041F1803231F54AD1AA20E9F08530D9F06E
:107CD00023D083FD18C082FFF7CF04C0A2DE8193BA
:107CE000615031F09091F3008091F200892BB1F74F
:107CF000D4DF611549F704C0AA2029F0853019F0B6
:107D00000BD080FFF9CF8EE79091E8008923809314
:107D1000E800089584E089DB8091E800089580916F
:107D2000E2000895FCDF8E7F80618093E200089579
:107D300082E061EC09D083E061E802D084E060E891
:107D400042E103C080E060E042E06FDB81E007D009
:107D50001092ED006093EC004093ED000895909137
:107D6000EB00892B8093EB00089560E0923029F0BE
:107D7000913029F4E0E062E102C0E2E16EE3F1E07B
:107D8000089580915B0188234CF402C0AA20C1F3BE
:107D9000C3DF82FFFBCF81CFAA2091F3BDDF80FF3D
:107DA000FBCFB1CF4091610150916201461751055F
:107DB00020F0462F611509F4A6DF50E022C0AA206A
:107DC00061F1853051F1A8DF83FD67CFA5DF82FD2A
:107DD00021C080FF16C03091F3002091F20006C050
:107DE00081918093F10041502F5F3F4F411519F071
:107DF00028303105A8F350E02830310509F451E06E
:107E000082DF4115E1F65523D1F604C0AA2029F0FE
:107E1000853019F081DF82FFF9CF3FCFEBE5F1E04C
:107E200000DE8193E336E1F73BDF76DF83FF91C02D
:107E300080915B0190915C01913009F170F0933079
:107E4000F1F0953009F444C0963009F456C09830EA
:107E500009F460C0993059F767C0823841F78091C2
:107E60005F01E2DA2091EB001092E90077D02295D1
:107E7000269521702093F1001092F10052C08823C2
:107E800011F08230A1F68F71823089F680915D0108
:107E90008823D1F420915F01277049F22093E900F3
:107EA0008091EB0080FF10C0933011F480E20BC092
:107EB00080E155DF81E0880F2A95E9F78093EA0099
:107EC0001092EA0088E04BDF1092E90047D02AC008
:107ED000882391F410915D0110680FB7F8943ED09B
:107EE00050DF1ADF80FFFDCF1093E300103883E0EE
:107EF00009F482E0A82E0FBF2CC08058823048F5CC
:107F000080915D0190915E0130DF603011F126D0EB
:107F100049DF1FC08038E9F421D08091530180935C
:107F2000F100F1DE2EDF15C0882399F490915D01F8
:107F3000923078F49093530111D023DF8091530154
:107F4000882321F48091E30091E087FD94E0A92E3D
:107F5000EFDEE2DE83FF089580E201DF87EFD4CE1B
:107F6000A3E6B1E0F437B8F40ED090E40D901D9084
:107F700081E087BFE89532969A95C1F71124E058C1
:107F8000F04085E001C083E001D081E187BFE89542
:087F900007B600FCFDCF0895C7
:067FFA003231B3CFFBDCC5
:040000030000740085
:00000001FF
